:100000000C9483000C94A4000C94A4000C94A40001
:100010000C94A4000C94A4000C94A4000C94A400D0
:100020000C94A4000C94A4000C94A4000C94A400C0
:100030000C94A4000C94A4000C94A4000C94A400B0
:100040000C94A4000C94A4000C94A4000C94A400A0
:100050000C94A4000C94A4000C94A4000C94A40090
:100060000C94A4000C94A6000C9456010C94A400CB
:100070000C94A4000C94A4000C94A4000C94A40070
:100080000C94A4000C94A4000C94A4000C94A40060
:100090000C94D2000C9482010C94A4000C943807A8
:1000A0000C94A4000C94A4000C94A4000C94A40040
:1000B0000C94A4000C94A4000C94A4000C94A40030
:1000C0000C94A4000C94A4000C94A4000C94FE00C6
:1000D0000C94AE010C94A4000C942A010C94DA0147
:1000E0000C94A40045464765666700202B2D2E30F2
:1000F00031323334353637383968006364696E6FAE
:1001000070737578580011241FBECFEFD1E2DEBFA7
:10011000CDBF00E00CBF12E0A0E0B2E0E6EBF4E2FD
:1001200000E00BBF02C007900D92A03BB107D9F7CA
:1001300012E0A0EBB2E001C01D92A03DB107E1F7D3
:100140000E9406020C9459120C9400001F920F9208
:100150000FB60F920BB60F9211242F933F934F932C
:100160005F936F937F938F939F93AF93BF93EF931F
:10017000FF938091B0029091B1020E94660AFF91B4
:10018000EF91BF91AF919F918F917F916F915F910F
:100190004F913F912F910F900BBE0F900FBE0F907C
:1001A0001F9018951F920F920FB60F920BB60F92D9
:1001B00011242F933F934F935F936F937F938F936C
:1001C0009F93AF93BF93EF93FF938091B20290916F
:1001D000B3020E94660AFF91EF91BF91AF919F9188
:1001E0008F917F916F915F914F913F912F910F90E0
:1001F0000BBE0F900FBE0F901F9018951F920F927D
:100200000FB60F920BB60F9211242F933F934F937B
:100210005F936F937F938F939F93AF93BF93EF936E
:10022000FF938091B4029091B5020E94660AFF91FB
:10023000EF91BF91AF919F918F917F916F915F915E
:100240004F913F912F910F900BBE0F900FBE0F90CB
:100250001F9018951F920F920FB60F920BB60F9228
:1002600011242F933F934F935F936F937F938F93BB
:100270009F93AF93BF93EF93FF938091B6029091BA
:10028000B7020E94660AFF91EF91BF91AF919F91D3
:100290008F917F916F915F914F913F912F910F902F
:1002A0000BBE0F900FBE0F901F9018951F920F92CC
:1002B0000FB60F920BB60F9211242F933F934F93CB
:1002C0005F936F937F938F939F93AF93BF93EF93BE
:1002D000FF938091B0029091B1020E94AD0AFF910C
:1002E000EF91BF91AF919F918F917F916F915F91AE
:1002F0004F913F912F910F900BBE0F900FBE0F901B
:100300001F9018951F920F920FB60F920BB60F9277
:1003100011242F933F934F935F936F937F938F930A
:100320009F93AF93BF93EF93FF938091B20290910D
:10033000B3020E94AD0AFF91EF91BF91AF919F91DF
:100340008F917F916F915F914F913F912F910F907E
:100350000BBE0F900FBE0F901F9018951F920F921B
:100360000FB60F920BB60F9211242F933F934F931A
:100370005F936F937F938F939F93AF93BF93EF930D
:10038000FF938091B4029091B5020E94AD0AFF9153
:10039000EF91BF91AF919F918F917F916F915F91FD
:1003A0004F913F912F910F900BBE0F900FBE0F906A
:1003B0001F9018951F920F920FB60F920BB60F92C7
:1003C00011242F933F934F935F936F937F938F935A
:1003D0009F93AF93BF93EF93FF938091B602909159
:1003E000B7020E94AD0AFF91EF91BF91AF919F912B
:1003F0008F917F916F915F914F913F912F910F90CE
:100400000BBE0F900FBE0F901F9018958F929F926A
:10041000AF92BF92CF92DF92EF92FF920F931F9312
:10042000DF93CF93CDB7DEB762970FB6F894DEBFF8
:100430000FBECDBF1AB81BB880E884B985B180580B
:1004400085B984E690E00E949E0885B1805885B900
:1004500084E690E00E949E0885B1805885B984E6C4
:1004600090E00E949E0885B1805885B984EF91E0A4
:100470000E949E0880E040E056E960E070E028E2DB
:1004800008E20E94FF089093B9028093B802789422
:100490006091B8027091B90280E092E00E948B11E5
:1004A00080E00E94D70400D000D0EDB7FEB73196AF
:1004B0002091B8023091B902ADB7BEB712963C9305
:1004C0002E9311972EE032E033832283992787FD04
:1004D0009095958384830E944E110091B8021091EB
:1004E000B9022DB73EB72A5F3F4F0FB6F8943EBF13
:1004F0000FBE2DBF0E94320700D000D0EDB7FEB76F
:100500003196ADB7BEB712961C930E9311972FE19B
:1005100032E03383228386958695848315820E94F8
:100520004E110091B8021091B9022DB73EB72A5F63
:100530003F4F0FB6F8943EBF0FBE2DBF0E94350748
:1005400000D000D0EDB7FEB73196ADB7BEB712966A
:100550001C930E9311972DE232E03383228386950C
:100560008695848315820E944E112DB73EB72A5F6F
:100570003F4F0FB6F8943EBF0FBE2DBF8091B8021B
:100580009091B9020E9468046E010894C11CD11CAC
:1005900023E4E22E22E0F22E08E512E097E0A92EF5
:1005A000B12CAC0EBD1E8DE0882E912C8C0E9D1EA4
:1005B0008091B8029091B9020E94FA0A8823C1F38F
:1005C0008091B8029091B9020E940C11873699F17E
:1005D000883618F4813661F706C08D3609F453C0A9
:1005E000833731F7ABC0C4010E941C06ADB7BEB75C
:1005F0001C970FB6F894BEBF0FBEADBFEDB7FEB7E8
:1006000031962091B8023091B90212963C932E9304
:100610001197F382E282992787FD909595838483D1
:100620008D859E85978386838F859889918780871E
:1006300089899A894FC0C6010E94AF05ADB7BEB780
:100640001C970FB6F894BEBF0FBEADBFEDB7FEB797
:1006500031962091B8023091B90212963C932E93B4
:100660001197F382E282992787FD90959583848381
:1006700089819A81978386838B819C8191878087EA
:100680008D819E8127C0C5010E947606ADB7BEB799
:100690001C970FB6F894BEBF0FBEADBFEDB7FEB747
:1006A00031962091B8023091B90212963C932E9364
:1006B0001197F382E282992787FD90959583848331
:1006C0008F8198859783868389859A85918780878E
:1006D0008B859C85938782870E944E112DB73EB7EC
:1006E000245F3F4F0FB6F8943EBF0FBE2DBF0E9450
:1006F000090618160CF05CCF00D000D0EDB7FEB79D
:1007000031962091B8023091B902ADB7BEB71296BA
:100710003C932E93119713830283992787FD90951D
:10072000958384830E944E112DB73EB72A5F3F4FB9
:100730000FB6F8943EBF0FBE2DBF3ACF8091B802DE
:100740009091B9020E94AF0433CF1F93DF93CF93F0
:100750000F92CDB7DEB7182F8091BE029091BF02E5
:1007600049830E943D0B8091BE029091BF02498156
:10077000642F0E943D0B812F62E040E00E948008C0
:100780000E9477089091C00281E09F3F09F480E0C9
:100790000F90CF91DF911F9108951F93182F809193
:1007A000BE029091BF020E943D0B812F61E041E0AB
:1007B0000E9480080E9477088091C0028F3F49F410
:1007C0008091BC029091BD020E94720B282F30E0F4
:1007D00002C02FEF3FEFC9011F9108950F931F93A0
:1007E000DF93CF930F920F92CDB7DEB7082F162F5E
:1007F0002A8349830E94CD032A81498197FD1CC029
:10080000222351F021E030E002C0220F331F4A952D
:10081000E2F7282B392B0BC021E030E002C0220F79
:10082000331F4A95E2F72095309528233923802FEE
:10083000612F422F0E94A5030F900F90CF91DF915F
:100840001F910F910895FF920F931F93DF93CF9302
:100850000F920F92CDB7DEB7F82E162F2F9A2A835C
:1008600049830E94CD032A81498197FD29C02F9891
:10087000A42FB0E01196A21BB109E1E0F0E002C0A4
:10088000EE0FFF1F2A95E2F731970A2E02C0EE0FF6
:10089000FF1F0A94E2F7F0E0AF014095509548231E
:1008A0005923802F90E002C0880F991FAA95E2F784
:1008B0008E239F23482B592B8F2D612F0E94A50338
:1008C0000F900F90CF91DF911F910F91FF9008959E
:1008D000CF93DF93EC018091BA0267E30E94CD03CE
:1008E00000D000D0EDB7FEB73196ADB7BEB71296C7
:1008F000DC93CE9311972BE632E0338322839583EA
:1009000084830E944E118DB79EB706960FB6F89459
:100910009EBF0FBE8DBF8091BA026AE60E94CD03D2
:1009200000D000D0EDB7FEB73196ADB7BEB7129686
:10093000DC93CE93119720E832E0338322839583B2
:1009400084830E944E118DB79EB706960FB6F89419
:100950009EBF0FBE8DBF80E0DF91CF910895CF93F2
:10096000DF93EC018091BC029091BD020E948C0B40
:1009700000D000D0EDB7FEB73196ADB7BEB7129636
:10098000DC93CE93119723E932E03383228395835E
:1009900084830E944E118DB79EB706960FB6F894C9
:1009A0009EBF0FBE8DBF80E0DF91CF9108950F9362
:1009B0008170982F9866990F9093BA028C60880F77
:1009C0008093BB02789480E160E10E944E088091A0
:1009D000BA026BE641E00E94A503882309F09AC0A1
:1009E0008091BA026BE144E022E001E00E9423041E
:1009F000882309F091C08091BA026CE144E022E0C2
:100A000000E00E942304882309F088C08091BA0284
:100A100064E240E40E94A503882309F081C080912C
:100A2000BA0265E24CE80E94A503882309F07AC067
:100A30008091BA0266E242E00E94A503882309F091
:100A400073C08091BA0267E248E80E94A503882338
:100A500009F06CC08091BA0268E24CE00E94A503E4
:100A6000882309F065C08091BA0269E24AE00E94D9
:100A7000A503882309F05EC08091BA026AE241E8CA
:100A80000E94A503882309F057C08091BA0264E64A
:100A900041E00E94A503882309F050C08091BA026A
:100AA00067E643E00E94A503882309F049C08091CE
:100AB000BA0264E344E00E94A503882309F042C01F
:100AC0008091BA0264E640E00E94A5038823E1F524
:100AD0008091BA026AE640E00E94A5038823B1F53E
:100AE0008091BA0264E641E00E94A503882381F563
:100AF0008091BA026AE640E20E94A503882351F57C
:100B00008091BA0264E343E10E94A503882321F1A6
:100B10008DED23C08FEF21C08EEF1FC08DEF1DC064
:100B20008CEE1BC08BEE19C08AEE17C089EE15C083
:100B300088EE13C087EE11C086EE0FC085EE0DC0A3
:100B400084EE0BC082EE09C081EE07C080EE05C0C6
:100B50008FED03C08EED01C080E00F9108951F93CB
:100B6000CF93DF93EC018091BE029091BF0263E4CA
:100B70000E943D0B8091BA0261E046E00E9480082D
:100B80000E9477088091C0028F3FF1F58091BC02EE
:100B90009091BD020E94720B182F8091BC0290911F
:100BA000BD020E94720B312F20E090E0822B932B2C
:100BB000998388838091BC029091BD020E94720B40
:100BC000182F8091BC029091BD020E94720B312FB0
:100BD00020E090E0822B932B9B838A838091BC0240
:100BE0009091BD020E94720B182F8091BC029091CF
:100BF000BD020E94720B312F20E090E0822B932BDC
:100C00009D838C8380E001C08FEFDF91CF911F9196
:100C100008951F938091BC029091BD020E948C0B9D
:100C2000182F181634F48091BC029091BD020E94D6
:100C30009A0B812F1F9108951F93CF93DF93EC019F
:100C40008091BE029091BF026BE30E943D0B8091A8
:100C5000BA0261E046E00E9480080E947708809115
:100C6000C0028F3FF1F58091BC029091BD020E94BD
:100C7000720B182F8091BC029091BD020E94720BE2
:100C8000312F20E090E0822B932B998388838091F1
:100C9000BC029091BD020E94720B182F8091BC0281
:100CA0009091BD020E94720B312F20E090E0822BC8
:100CB000932B9B838A838091BC029091BD020E94FA
:100CC000720B182F8091BC029091BD020E94720B92
:100CD000312F20E090E0822B932B9D838C8380E04A
:100CE00001C08FEFDF91CF911F9108951F93CF9394
:100CF000DF93EC018091BE029091BF026AE40E94F2
:100D00003D0B8091BA0261E046E00E9480080E949B
:100D100077088091C0028F3F09F041C08091BC02EA
:100D20009091BD020E94720B182F8091BC0290918D
:100D3000BD020E94720B382F20E0812F90E0822BA1
:100D4000932B998388838091BC029091BD020E946D
:100D5000720B182F8091BC029091BD020E94720B01
:100D6000382F20E0812F90E0822B932B9B838A8366
:100D70008091BC029091BD020E94720B182F80914D
:100D8000BC029091BD020E94720B382F20E0812F8F
:100D900090E0822B932B9D838C8380E001C08FEFAA
:100DA000DF91CF911F9108951F93CF93DF93EC01B3
:100DB0008091BE029091BF0263E00E943D0B809142
:100DC000BB0261E046E00E9480080E9477088091A3
:100DD000C0028F3F09F041C08091BC029091BD02DA
:100DE0000E94720B182F8091BC029091BD020E944C
:100DF000720B382F20E0812F90E0822B932B998368
:100E000088838091BC029091BD020E94720B182FC2
:100E10008091BC029091BD020E94720B382F20E09D
:100E2000812F90E0822B932B9B838A838091BC023D
:100E30009091BD020E94720B182F8091BC0290917C
:100E4000BD020E94720B382F20E0812F90E0822B90
:100E5000932B9D838C8380E001C08FEFDF91CF9136
:100E60001F9108958091BA0208958091BB02089560
:100E70001F920F920FB60F920BB60F9211241F9371
:100E80002F933F934F935F936F937F938F939F9392
:100E9000AF93BF93EF93FF938091C002833009F427
:100EA00052C0843034F4882351F0813009F0E2C01C
:100EB00023C08430A9F1853009F0DCC0A4C0809142
:100EC000B900887F883011F0803191F48091C2029E
:100ED000882339F084E08093C0028091C3028E7F22
:100EE000BFC081E08093C0028091C3028160B8C01E
:100EF0009EEF9093C0024BC01091B900187F103440
:100F0000D1F48091C102813011F480E001C080E40D
:100F10000E94F70883E08093C0021092C4026DC063
:100F20001091B900187F183131F41092C40285E095
:100F30008093C00285C08EEF8093C0020E94E008BB
:100F40001093C50297C08091B900887F883511F54C
:100F50008091BC029091BD020E948C0BE091BC027A
:100F6000F091BD02228133812150304082179307D6
:100F700031F06091BB00CF010E943D0B02C0809117
:100F8000BB008FEF8093C0020E94E00888E5809349
:100F9000C50270C0803561F58091BC029091BD02A0
:100FA0000E948C0BE091BC02F091BD022281338142
:100FB000215030408217930731F06091BB00CF0180
:100FC0000E943D0B02C08091BB002091C4022F5FA4
:100FD0002093C4028091C10230E090E0019728176D
:100FE000390711F480E001C080E40E94F70805C0D1
:100FF0009EEF9093C0028093C5028091BC008068F0
:101000008093BC0037C08091B900887F883259F541
:101010008091C4028F5F8093C4029091C2028917AD
:1010200079F48091C102882339F01092C0021092A5
:10103000C2020E94D0081EC08FEF8093C00218C069
:101040008091BE029091BF02FC01448155812681AE
:1010500037814217530711F48AE502C00E94720BD0
:101060000E94D70807C09EEF9093C0028093C502EC
:101070000E94E008FF91EF91BF91AF919F918F91F6
:101080007F916F915F914F913F912F911F910F90A1
:101090000BBE0F900FBE0F901F901895DF93CF934C
:1010A0000F92CDB7DEB790E069830E94060B909354
:1010B000BD028093BC026981862F90E00E94060BDE
:1010C0009093BF028093BE0284E08093BC008FEFB8
:1010D0008093C00288E18093B80080E00E94E70816
:1010E00081E00E94EF080F90CF91DF9108958091E9
:1010F000C00287FFFCCF8091BC0084FDF8CF08952B
:10110000DF93CF9300D0CDB7DEB74B836A8389835B
:101110000E9477081092C00289818093C3024B819C
:101120004093C1026A816093C2020E94D00881E0AC
:101130000F900F900F90CF91DF910895EF92FF9253
:101140000F931F93BC0180E090E020EA3FE040E075
:1011500050E00E94130F9B01AC017A0100E010E007
:1011600080E090E0DC0160E070E006C0FB013197B8
:10117000F1F70196A11DB11D8E159F05A007B107BE
:10118000A8F340705070211531054105510519F043
:10119000C9010197F1F71F910F91FF90EF9008950A
:1011A000ECEBF0E080818174846A80830895809301
:1011B000BB00ECEBF0E0808181748468808308954B
:1011C000ECEBF0E080818174846980830895E9EB21
:1011D000F0E0908183709C7F892B80830895ECEBF5
:1011E000F0E0908181709E7F892B80830895ECEBE5
:1011F000F0E0908180749F73892B808308956F92B3
:101200007F928F929F92AF92BF92CF92DF92FF9286
:101210000F931F93DF93CF930F92CDB7DEB7F82EC6
:101220005A016B01223008F4ABC0013009F4A8C0A8
:1012300089E090E029830E947B0F3C01FC01F08251
:10124000298121830283148284818383168286818B
:101250008583822F90E0800F911D0E947B0F8C016F
:10126000F30190878783A601950184E0220F331F45
:10127000441F551F8A95D1F760E074E284EF90E037
:101280000E94590F21503040FF2DF13011F1F13003
:1012900030F0F230C1F1F33009F069C04EC088E19E
:1012A0008093C1003093C5002093C40082ED99E083
:1012B0006CE47AE00E94C110FC017586648670922D
:1012C000B1026092B0028091C10080688093C10039
:1012D00059C088E18093C9003093CD002093CC00A1
:1012E00082ED99E06CE47AE00E94C110FC01758601
:1012F00064867092B3026092B2028091C9008068E5
:101300008093C9003FC088E18093D1003093D5001D
:101310002093D40082ED99E06CE47AE00E94C11041
:10132000FC01758664867092B5026092B402809169
:10133000D10080688093D10025C088E1809331017D
:10134000309335012093340182ED99E06CE47AE02A
:101350000E94C110FC01758664867092B70260928B
:10136000B602809131018068809331010BC0011574
:10137000110519F0C8010E941510C3010E94151033
:10138000E0E0F0E0CF010F90CF91DF911F910F913E
:10139000FF90DF90CF90BF90AF909F908F907F9005
:1013A0006F900895CF93DF93482FDB011C96ED914A
:1013B000FC911D972281223008F444C030E0E901FD
:1013C000219786815581B901680F711DCB01851B5D
:1013D0009109B9010E94460F8C179D0791F39681E0
:1013E0008181A781B085A90FB11DA80FB11D4C93B4
:1013F000868190E00196628170E00E94460F8683AC
:101400008081813069F0813028F0823079F083303A
:10141000F1F512C08091C10080628093C10037C095
:101420008091C90080628093C90031C08091D10051
:1014300080628093D1002BC08091310180628093C3
:10144000310125C08081813071F0813028F08230F7
:1014500089F08330E1F415C08091C00085FFFCCF96
:101460004093C60014C08091C80085FFFCCF409314
:10147000CE000DC08091D00085FFFCCF4093D600F8
:1014800006C08091300185FFFCCF4093360180E09B
:1014900090E0DF91CF910895DC011C96ED91FC91D5
:1014A0001D97938184819817E1F38381A781B0858B
:1014B000A80FB11D2C91838190E00196618170E0AD
:1014C0000E94460F8383822F90E00895FC01808163
:1014D000813071F0813028F0823089F08330E1F47E
:1014E00015C08091C00087FF37C04091C60014C06E
:1014F0008091C80087FF30C04091CE000DC0809120
:10150000D00087FF29C04091D60006C080913001ED
:1015100087FF22C040913601218130E084815381D0
:10152000B901680F711DCB01851B9109B9010E949A
:10153000460F215030408217930774F48481A781AD
:10154000B085A80FB11D4C93848190E00196618114
:1015500070E00E94460F84830895FC019581868186
:101560002081981709F5213069F0213028F02230C8
:1015700079F02330F1F512C08091C1008F7D809306
:10158000C10008958091C9008F7D8093C90008959E
:101590008091D1008F7D8093D10008958091310199
:1015A0008F7D80933101089585819181A781B085D8
:1015B000A90FB11DA80FB11D3C91858190E0019646
:1015C000628170E00E94460F8583213051F0213006
:1015D00028F0223049F0233061F409C03093C6006E
:1015E00008953093CE0008953093D6000895309337
:1015F00036010895DC011C96ED91FC911D97238125
:10160000948181E0291709F480E00895CF92DF9258
:10161000EF92FF920F931F93CF93DF938C0188E09B
:1016200090E00E947B0F7C01C82EE6016E01DF2C4A
:10163000E6012097C1F00115110539F0C8010E949B
:101640007B0F99838883009731F4C7010E9415109E
:10165000C0E0D0E008C01B830A831F821E828E81F7
:101660009F819D838C83CE01DF91CF911F910F913C
:10167000FF90EF90DF90CF9008950F931F93DF932B
:10168000CF930F92CDB7DEB78C01C80169830E945A
:101690008C0BD80112962D913C911397215030401C
:1016A00069818217930789F316968D919C911797FC
:1016B000ED91FC911197E80FF91F608316968D91BB
:1016C0009C911797019612966D917C9113970E94A9
:1016D000320FF801978386830F90CF91DF911F918E
:1016E0000F910895FC012481358186819781281707
:1016F0003907C9F384819581A081B181A80FB91FF1
:101700004C91848195810196628173810E94320F90
:1017100095838483842F0895FC016281738186817F
:10172000978124813581860F971F821B930B0E941E
:10173000320F0895CF93DF93EC0103C0CE010E94D6
:10174000720B2C813D818E819F8128173907B1F75B
:10175000DF91CF9108956F927F928F929F92AF9277
:10176000BF92CF92DF92EF92FF920F931F93DF937E
:10177000CF93CDB7DEB72C970FB6F894DEBF0FBE70
:10178000CDBF6C013B018A01FC0117821682838167
:1017900081FD03C01EC1850104C04E010894811C57
:1017A000911CF601E380F301E3FC8591E3FE819156
:1017B0003F01882309F409C1853251F4E3FC2591E6
:1017C000E3FE21913F01253211F0FF2423C085E281
:1017D00090E0B6010E945F115801DDCF222309F489
:1017E00089C08BEE90E0622F70E02C870E94B610CB
:1017F0002C85009749F4233219F4F0E1FF2A04C044
:101800002C3669F420E8F22AF301E3FC2591E3FE8B
:1018100021913F01F7FEE2CF222309F43FC084EE7D
:1018200090E0622F70E02C870E94B6102C85009704
:1018300041F064E0A62EB12CA00EB11E8FE390E023
:101840000FC0233629F0233789F0233529F50CC042
:1018500052E0A52EB12CA00EB11EF801808191811D
:10186000B6010E945F1197CFF1E0FF2A42E0A42E5B
:10187000B12CA00EB11EF8010081118104C090E0CE
:10188000B6010E945F11F801F0FC8591F0FE819194
:101890008F018823A1F77FCF243611F0293651F527
:1018A000F7FE0BC034E0A32EB12CA00EB11EF80140
:1018B00060817181828193810CC022E0A22EB12CC3
:1018C000A00EB11EF80160817181882777FD809597
:1018D000982FFFEEFF2297FF09C090958095709595
:1018E00061957F4F8F4F9F4F20E4F22AA4012AE099
:1018F00030E03BC0203799F0213730F42835B1F083
:101900002F3609F062C017C0253721F0283709F0BB
:101910005CC007C08FEEF8222AE030E00EC0E0E1A4
:10192000FE2AF4E2FF2A20E130E007C024E0F22A98
:1019300020E132E002C028E030E0F7FE0BC094E086
:10194000A92EB12CA00EB11EF80160817181828197
:1019500093810AC082E0A82EB12CA00EB11EF8011E
:101960006081718180E090E0A4010E94CC11E82E9A
:10197000E8180F2D10E0F6FE05C08DE290E0B601EC
:101980000E945F1104FF15C0FE01EE0DF11D808164
:10199000803379F080E390E0B6010E945F1102FF8E
:1019A00008C0C80180729070885A9F4FB6010E948B
:1019B0005F11EA94F401EE0DF11D808190E0B60113
:1019C0000E945F11EE20A9F7E6CEF601268137814D
:1019D00002C02FEF3FEFC9012C960FB6F894DEBF7F
:1019E0000FBECDBFCF91DF911F910F91FF90EF9070
:1019F000DF90CF90BF90AF909F908F907F906F902F
:101A0000089520FD09C0FC0123FD05C022FF02C08E
:101A100073836283518340830895EF92FF920F9303
:101A20001F9344FD10C046FD10C0DB01FC01AA0F4E
:101A3000BB1FEE1FFF1F1094D1F76A0F7B1F8E1F75
:101A40009F1F31E003C033E001C034E0660F771F11
:101A5000881F991F3150D1F77B018C01E20EF11CD8
:101A6000011D111DA8019701B701CA011F910F9116
:101A7000FF90EF900895EF92FF920F931F93CF93F3
:101A8000DF938C01C8010E940C11EC0197FD08C086
:101A90000E94AE100097B1F7CE01B8010E94B111BB
:101AA000CE01DF91CF911F910F91FF90EF9008959C
:101AB0008F929F92AF92BF92DF92EF92FF920F931D
:101AC0001F93DF93CF930F92CDB7DEB74C01D62E85
:101AD0005A01122F0E940C118B3219F08D3249F4E9
:101AE0001068DA9409F46CC0C4010E940C1197FDCF
:101AF00067C0312F3D7F232F2073F1F48033E1F451
:101B0000DA9409F448C0C40139830E940C11398168
:101B100097FD41C03260883711F0883559F4306440
:101B2000DA94C9F1C40139830E940C11398197FFFD
:101B300003C031C036FF3061EE24FF248701282F17
:101B40002053283090F034FD09C02A3070F036FF61
:101B500005C02F7D422F4151463030F0B40139830A
:101B60000E94B111398114C02750C801B701432F19
:101B700039830E940D0D7B018C0139813260DA942A
:101B800069F0C40139830E940C11398197FFD7CFC6
:101B900031FD04C015C0EE24FF24870137FF08C0C3
:101BA00010950095F094E094E11CF11C011D111DAD
:101BB000C501B801A701232F0E94010D81E001C0DA
:101BC00080E00F90CF91DF911F910F91FF90EF90E8
:101BD000DF90BF90AF909F908F9008954F925F924B
:101BE0006F927F929F92AF92BF92CF92DF92EF92CD
:101BF000FF920F931F93DF93CF930F92CDB7DEB772
:101C00008C015B013A01FC0117821682EE24E6C0CA
:101C10008F2D90E00E94AE10009721F0C8010E9425
:101C20003B0DDCC0FF2DF53251F4F501C3FC3591BD
:101C3000C3FE31915F01353271F455E2F52EC801D2
:101C40000E940C1197FDD6C0F81609F4C7C0B80160
:101C50000E94B111D1C03A3241F4C3FC3591C3FEA8
:101C600031915F01FF24F39401C0FF24992410C037
:101C7000F2E0FF2A692D70E080E090E040E20E94EF
:101C80000D0D962EF501C3FC3591C3FE31915F0118
:101C9000232F20532A3060F3F1FE03C0992019F45A
:101CA000ABC099249A94383619F03C3699F40AC09E
:101CB000F501C3FC3591C3FE31915F01383651F413
:101CC000F8E0FF2A44E0F42AF501C3FC3591C3FE95
:101CD00031915F01332309F48FC08BEF90E0632FC4
:101CE00070E039830E94B6103981009709F484C0EE
:101CF0008F2DF0FC08C0F3014080518042E050E09D
:101D0000640E751E02C0442455243E3651F4F80179
:101D10004681578160E070E0C2012F2D0E94010DC5
:101D20005DC0333691F481FD02C099249394C801BB
:101D30000E940C1197FD5EC04114510419F0F2018C
:101D400081932F019A9499F747C0C80139830E9463
:101D50003B0D398197FD4EC03F3661F1303728F495
:101D6000343629F1393649F52AC0333719F0353779
:101D700021F51DC0C8010E940C116C0197FD11C016
:101D80000E94AE10009729F0C601B8010E94B1115F
:101D900008C04114510419F0F201C1922F019A9424
:101DA00049F741145104C1F0F201108215C0F0E26C
:101DB000FF2A05C040E1F42A02C050E4F52AC80118
:101DC000692DA2012F2D0E94580D882329F4F801B6
:101DD0008381807379F410C0F0FEE394F801C3802E
:101DE000F501C3FCF590C3FEF1905F01FF2009F0FF
:101DF0000FCF02C0EE2019F02E2D30E002C02FEFE1
:101E00003FEFC9010F90CF91DF911F910F91FF908C
:101E1000EF90DF90CF90BF90AF909F907F906F90AA
:101E20005F904F900895629FD001739FF001829F51
:101E3000E00DF11D649FE00DF11D929FF00D839F59
:101E4000F00D749FF00D659FF00D9927729FB00DF6
:101E5000E11DF91F639FB00DE11DF91FBD01CF0109
:101E600011240895AA1BBB1B51E107C0AA1FBB1F69
:101E7000A617B70710F0A61BB70B881F991F5A9516
:101E8000A9F780959095BC01CD01089597FB092E87
:101E900007260AD077FD04D0E5DF06D000201AF42B
:101EA000709561957F4F0895F6F7909581959F4FB6
:101EB0000895A1E21A2EAA1BBB1BFD010DC0AA1F8B
:101EC000BB1FEE1FFF1FA217B307E407F50720F0A3
:101ED000A21BB30BE40BF50B661F771F881F991F1E
:101EE0001A9469F760957095809590959B01AC0167
:101EF000BD01CF010895CF93DF938230910510F497
:101F000082E090E0E091C802F091C90240E050E028
:101F100020E030E026C06081718168177907E0F029
:101F20006817790781F4828193812115310531F099
:101F3000D90113969C938E9312972BC09093C9024C
:101F40008093C80226C04115510519F06417750722
:101F500018F4AB01E901DF019F0172816381E72F72
:101F6000F62F3097C1F64115510501F1481B590B69
:101F70004430510580F412968D919C9113972097CF
:101F800019F09B838A8304C09093C9028093C8028E
:101F9000FD01329646C0FD01E40FF51F8193919338
:101FA0004250504011965C934E933BC02091C60224
:101FB0003091C7022115310541F42091AB023091D7
:101FC000AC023093C7022093C6022091AD0230913B
:101FD000AE022115310541F42DB73EB74091A9025B
:101FE0005091AA02241B350BE091C602F091C70262
:101FF000E217F307A0F42E1B3F0B2817390778F0E0
:10200000AC014E5F5F4F2417350748F04E0F5F1F3E
:102010005093C7024093C6028193919302C0E0E0BF
:10202000F0E0CF01DF91CF910895CF93DF93009738
:1020300009F491C0FC013297138212826091C802A8
:102040007091C9026115710581F420813181280FD9
:10205000391F8091C6029091C7028217930799F5A4
:10206000F093C702E093C60276C0DB0180E090E007
:1020700002C0CD01D901AE17BF0748F412962D91C9
:102080003C91139721153105A1F7CD0121C0B383F0
:10209000A283EF01499159919E01240F351FA21788
:1020A000B30779F42D913C911197240F351F2E5FC2
:1020B0003F4F3183208312962D913C9113973383A8
:1020C0002283009729F4F093C902E093C80243C029
:1020D000DC011396FC93EE9312974D915D91A40F42
:1020E000B51FEA17FB0769F420813181240F351FE2
:1020F0002E5F3F4FEC0139832883228133813B835C
:102100002A83E0E0F0E002C0FB01BC01DB01129693
:102110008D919C9113970097B9F79B012E5F3F4FCC
:102120008D919C911197820F931F4091C6025091FF
:10213000C7024817590779F4309729F41092C90259
:102140001092C80202C01382128222503040309393
:10215000C7022093C602DF91CF91089591119FC1CC
:10216000803219F089508550D0F70895FC01059010
:10217000061621F00020D9F7C00108953197CF014C
:1021800008950F931F93CF93DF938C01EB0100977A
:1021900011F42097C9F181E090E06EE070E00E94B8
:1021A0002A12FC019C01009789F180E88383209723
:1021B00071F0D387C28781E883838091CA029091AE
:1021C000CB02009721F4F093CB02E093CA020115F1
:1021D0001105E1F0118700878381826083838091FC
:1021E000CC029091CD02009789F4F093CD02E09358
:1021F000CC028091CE029091CF02009739F4F093F7
:10220000CF02E093CE0202C020E030E0C901DF91AE
:10221000CF911F910F910895CF93DF93EC013B81F4
:1022200030FF36C036FF09C03F7B3B838E819F81E4
:1022300001969F838E832A8129C032FF0FC0E881D7
:10224000F9818081992787FD9095009719F4306274
:102250003B831EC03196F983E88311C0EA85FB8574
:10226000CE01199597FF0BC02B813FEF8F3F93074E
:1022700011F480E101C080E2822B8B8309C02E81A2
:102280003F812F5F3F4F3F832E83282F30E002C0D6
:102290002FEF3FEFC901DF91CF910895DF93CF93E7
:1022A000CDB7DEB79E01265F3F4F8E819F81688547
:1022B0007985A9010E94AB0BCF91DF9108950F930F
:1022C0001F93CF93DF938C01EB018B8181FF1BC0A8
:1022D00082FF0DC02E813F818C819D812817390797
:1022E00064F4E881F9810193F983E88306C0E88505
:1022F000F985802F1995009731F48E819F81019681
:102300009F838E8302C00FEF1FEFC801DF91CF9133
:102310001F910F910895EF92FF920F931F93CF9308
:10232000DF937C01EB018B8181FF11C000E010E0A5
:1023300008C0E885F985BE011995009711F00FEFE7
:102340001FEFF70181917F01882399F702C00FEFFA
:102350001FEFC801DF91CF911F910F91FF90EF9078
:102360000895FB01238120FF13C026FD11C03FEF1C
:102370008F3F930769F0828320642F7D238326811A
:1023800037812150304037832683282F30E002C028
:102390002FEF3FEFC9010895FA01AA27283051F124
:1023A000203181F1E8946F936E7F6E5F7F4F8F4F86
:1023B0009F4FAF4FB1E03ED0B4E03CD0670F781FE5
:1023C000891F9A1FA11D680F791F8A1F911DA11DCA
:1023D0006A0F711D811D911DA11D20D009F4689403
:1023E0003F912AE0269F11243019305D3193DEF6AB
:1023F000CF010895462F4770405D4193B3E00FD061
:10240000C9F7F6CF462F4F70405D4A3318F0495D4B
:1024100031FD4052419302D0A9F7EACFB4E0A6952E
:102420009795879577956795BA95C9F70097610550
:10243000710508959B01AC010A2E069457954795A6
:1024400037952795BA95C9F7620F731F841F951F9B
:10245000A01D0895EF92FF920F931F93CF93DF93E8
:10246000689F8001699F100D789F100D1124C8018D
:102470000E947B0FE82EE7017E01F92EE7012097ED
:1024800031F08E2D60E070E0A8010E945212CE0162
:10249000DF91CF911F910F91FF90EF9008959927B1
:1024A00088270895DC0101C06D9341505040E0F74A
:0624B0000895F894FFCF2F
:1024B60068656C6C6F20776F726C640A0D00496EEC
:1024C600697469616C697A653A2025640A0D004170
:1024D6006464726573733A2025780A0D00436F6D44
:1024E6007061737320616464726573733A20257832
:1024F6000A0D0025643A20253036642025303664DE
:1025060020253036640A0D00466C757368656420B4
:1025160025642062797465730A0D0052415F494E45
:10252600545F50494E5F4346473A2025780A0D00CE
:1025360052415F555345525F4354524C3A202578D9
:102546000A0D00427974657320696E2062756666AD
:1025560065723A2025640A0D002000D002000000B2
:00000001FF
